
 Start  Stop   Length Name                   Class
 00000H 07D02H 07D03H DXDATA                 DATA
 07D10H 07F31H 00222H DXSTACK                STACK
 07F40H 0A786H 02847H DXCODE                 CODE
 0A790H 1067FH 05EF0H DXPMCODE               PMCODE

 Origin   Group
 0000:0   DGROUP

  Address         Publics by Name

 0000:799D       A20ENABLECOUNT
 0A79:3765       ADDSELECTORTOCHAIN
 0A79:3641       ADDTOXMEMHEAP
 0A79:042D       ALLOCATEEXCEPTIONSTACK
 07F4:207F       ALLOCATEEXTMEM
 0A79:3370       ALLOCATELDTSELECTOR
 0A79:3845       ALLOCATELOWBLOCK
 0A79:3378       ALLOCATESELECTOR
 0A79:33AB       ALLOCATESELECTORBLOCK
 0A79:37A4       ALLOCATEXMEM32
 0A79:3A4E       ALLOCATEXMEMBLOCK
 07F4:02D7       BACKFROMDOS
 0000:7BD0       BDMASERVICEBIT
 0000:4712       BPGDT
 0000:4714       BPGDTBASE
 0000:4712       BPGDTCB
 0000:471E       BPIDT
 0000:4720       BPIDTBASE
 0000:471E       BPIDTCB
 0000:4724       BPRMIVT
 0000:0100       BREFLSTACK
 0A79:3DEB       CALCULATEMAXIMUMSEGMENTSPACE
 0A79:3E39       CALCULATEMAXIMUMSPACE
 0000:7A52       CBHEAPSIZE
 0000:796C       CDPMICLIENTS
 0000:470A       CDSCGDTMAX
 0000:4718       CDSCIDTMAX
 07F4:2661       CHECKCPUTYPE
 0A79:108D       CHECKSTATUS
 07F4:0222       CHILDTERMINATIONHANDLER
 0000:7A40       CKBINITIALHEAPSIZE
 0000:6914       CLPRELOCITEM
 07F4:1700       CODEEND
 0A79:5EF0       CODEENDPM
 0A79:3EAD       COMBINEFREEBLOCKS
 0A79:5AE9       COPYBUFFER
 0A79:5ABF       COPYBUFFEROUT
 0A79:4D63       DD_I31_CLEAR_WATCHPOINT
 0A79:4DD7       DD_I31_GET_STATUS
 0A79:4E10       DD_I31_RESET_WATCHPOINT
 0A79:4CA7       DD_I31_SET_WATCHPOINT
 0000:7B80       DEBUG_REGS
 0A79:59DF       DELAYNETPOSTING
 0A79:5BD7       DELINK
 07F4:02BE       DETERMINEFREEMEMORY
 0A79:1196       DFGETINTRVECTOR
 0A79:11BC       DFSETINTRVECTOR
 07F4:02A1       DISPLAYERRORMSG
 0A79:40BE       DISPOSEBLOCK
 0A79:08C4       DOSENTRY
 0A79:0A14       DOSEXIT
 0A79:0DCD       DOSEXITCALL
 0A79:10B9       DOSXEC
 0A79:08C3       DOSXIRET
 07F4:0141       DOSXTERMINATIONHANDLER
 0000:7974       DPMIFLAGS
 0000:7972       DPMISEGATTR
 0A79:2C40       DPMISIZEINIT
 07F4:0DD0       DPMI_CLIENT_PMODE_ENTRY
 0000:7A42       DSEGCURRENT
 0000:4740       DTAOFFSET
 0000:473C       DTASEGMENT
 0000:473E       DTASELECTOR
 0A79:3522       DUPSEGMENTDSCR
 0A79:0006       DXPMINIT
 07F4:1AAF       EMMDISABLE
 07F4:1550       EMMENABLE
 0A79:5EEC       ENDNPXEXCEPTIONHANDLER
 07F4:0982       ENDRMINTRENTRY
 0A79:1D53       ENTERINTHANDLER
 07F4:0F90       ENTERPROTECTEDMODE
 07F4:1025       ENTERREALMODE
 07F4:1700       ER_CPUTYPE
 07F4:1895       ER_DXINIT
 07F4:1971       ER_EXTMEM
 07F4:19DA       ER_NOEXE
 07F4:17FD       ER_NOHIMEM
 07F4:176E       ER_PROTMODE
 07F4:1904       ER_REALMEM
 0000:6904       EXEC_PAR_BLK
 0000:474D       EXITCODE
 0000:79A1       F286_287
 0A79:336C       FARPARATOLDTSELECTOR
 0000:79A8       FASTBOP
 0000:7CD9       FASTERMODESWITCH
 0000:7C90       FDEBUG
 0000:474C       FFAULTABORT
 0000:73E6       FHARDWAREINTMOVED
 0000:6912       FHEXEFILE
 07F4:1DEC       FINDFILE
 0A79:3F10       FINDFREEBLOCK
 0A79:34CA       FINDLOWSELECTOR
 0A79:34DB       FINDSELECTOR
 0A79:5C0F       FINDTARGETNCB
 0000:7BC0       FMEMM_DISABLED
 0A79:290F       FNABORT
 0A79:2903       FNQUERYDOSEXTENDER
 0A79:39B2       FREELOWBLOCK
 0A79:4212       FREEMEMBYOWNER
 0A79:347A       FREESELECTOR
 0A79:34B9       FREESELECTORBLOCK
 0A79:3F9B       FREESPACE
 0A79:37C7       FREEXMEM32
 0A79:3BD4       FREEXMEMBLOCK
 0000:4750       FUSINGHMA
 0000:7CEB       FWIN30COMMDRV
 0A79:1049       GETENTRYCD
 0A79:5C52       GETENTRYEXITFLAGS
 07F4:1EF4       GETENV
 07F4:276C       GETEXENAME
 0A79:3080       GETFAULTVECTOR
 0A79:2F8B       GETINTRVECTOR
 0A79:313C       GETSEGMENTADDRESS
 07F4:02D6       GOINGTODOS
 0A79:0F09       GTAREA
 0A79:30DB       GTPARA
 0A79:5CB0       HANDLENETBIOSANR
 0000:7BE4       HCB_LIST
 0000:477D       HIGHESTDXSEL
 0000:79A6       HIGHESTSEL
 0000:474A       HMEMDOSX
 0000:7A44       HMEMHEAP
 0000:7A8D       HMEM_XMS_COUNT
 0000:7A6D       HMEM_XMS_TABLE
 0A79:5D95       HOOKNETBIOSHWINT
 0000:7AA0       I31HWRESET
 0A79:4914       I31_ALLOCCALLBACK
 0A79:46D2       I31_ALLOCDOSMEM
 0A79:4AB9       I31_ALLOCMEM
 0A79:446E       I31_ALLOCSEL
 0A79:45D5       I31_CREATEDATAALIAS
 0A79:4976       I31_FREECALLBACK
 0A79:4706       I31_FREEDOSMEM
 0A79:4AF9       I31_FREEMEM
 0A79:44A7       I31_FREESEL
 0A79:4A8E       I31_GETFREEMEM
 0A79:4E9B       I31_GETRAWMODESWITCH
 0A79:4514       I31_GETSEGADDR
 0A79:450C       I31_GETSELINCR
 0A79:460B       I31_GETSETDESCRIPTOR
 0A79:47CC       I31_GETSETFAULTVECTOR
 0A79:47FD       I31_GETSETPMINT
 0A79:4731       I31_GETSETRMINT
 0A79:4E67       I31_GETSTATESAVERESTORE
 0A79:44F9       I31_MAPSEG2SEL
 0A79:4BA3       I31_MEMGETHEADER
 0A79:4462       I31_PAGESIZE
 0A79:483F       I31_RMCALL
 0000:7AAB       I31_SELECTORBITMAP
 0A79:45A6       I31_SETACCESS
 0A79:455C       I31_SETLIMIT
 0A79:453A       I31_SETSEGADDR
 0A79:4724       I31_SIZEDOSMEM
 0A79:4B29       I31_SIZEMEM
 0A79:46AB       I31_SPECIFICSEL
 0A79:4460       I31_SUCCESS
 0A79:4B8B       I31_VERSION
 0A79:4B6B       I31_VIRTUALINT
 0A79:4ECA       I31_WOW_ALLOCSEL
 0A79:4F03       I31_WOW_SETALLOCFUNCTIONS
 0A79:4EE8       I31_WOW_SETDESCRIPTOR
 0000:4732       IDCPUTYPE
 07F4:1F50       INITDOSEXTENDER
 07F4:2285       INITGLOBALDSCRTABLE
 0A79:5DC0       INITIALIZEOEM
 07F4:249B       INITINTRDSCRTABLE
 0A79:3640       INITLOWHEAP
 0A79:55D0       INITNETMAPPER
 07F4:263D       INITTASKSTATESEG
 0A79:36C8       INITXMEMHEAP
 0000:7CC6       INT28FILTER
 0A79:5004       INTENTRY13
 0A79:51ED       INTENTRY2X
 0A79:1C08       INTENTRYMISC
 0A79:1CBE       INTENTRYMOUSE
 0A79:1AF4       INTENTRYVIDEO
 0A79:503E       INTEXIT13
 0A79:5217       INTEXIT2X
 0A79:1C27       INTEXITMISC
 0A79:1D20       INTEXITMOUSE
 0A79:1B48       INTEXITVIDEO
 0A79:0B1A       IOCTLENTER
 0A79:0CD0       IOCTLEXIT
 0A79:3463       ISSELECTORFREE
 07F4:10C8       LCODESEGLOC
 0A79:0894       LEAVEDOSEXTENDER
 0A79:1DD1       LEAVEINTHANDLER
 0A79:312E       LMA2SEGOFF
 0000:7CFB       LMADXPMCODE
 0000:7CF7       LMAGDT
 0000:7CF3       LMAIDT
 0000:7A90       LOWMEMALLOCFN
 0000:7A94       LOWMEMFREEFN
 0000:6BD4       LPFNUSERMOUSEHANDLER
 0000:6BDA       LPFNUSERPOINTINGHANDLER
 0000:472E       LPFNXMSFUNC
 0A79:35CF       MAKELOWSEGMENT
 0000:7BC2       MEMM_CALL
 0000:7BC1       MEMM_STATE
 0A79:3C64       MODIFYXMEMBLOCK
 07F4:0C1B       MOUSEINTERRUPTHANDLER
 0A79:09AE       MOVDAT
 07F4:2183       MOVEDOSEXTENDER
 07F4:21EF       MOVEDSCRTABLES
 0A79:35F9       MOVEMEMBLOCK
 0A79:0E7B       NET5FENTER
 0A79:0EAE       NET5FEXIT
 0A79:5911       NETBIOSPOSTROUTINE
 0000:7CB8       NETHEAPSIZE
 0A79:329F       NMOVEDESCRIPTOR
 0000:7A8F       NOASYNCSWITCHING
 0000:4706       NPEHSTACKLET
 0000:4704       NPEHSTACKLIMIT
 0A79:5E30       NPXEXCEPTIONHANDLER
 0000:6800       NPXFRBUF0
 0000:6802       NPXFRBUF1
 0A79:31A1       NSETSEGMENTACCESS
 0A79:3244       NSETSEGMENTBASE
 0A79:3545       NSETSEGMENTDSCR
 0A79:31FC       NSETSEGMENTLIMIT
 0A79:3313       NWOWSETDESCRIPTOR
 0A79:3355       PARATOLDTSELECTOR
 0A79:35EE       PARATOLINEAR
 07F4:2799       PARSECOMMANDLINE
 0000:4700       PBHWINTRSTACK
 0000:4702       PBREFLSTACK
 0000:6916       PLPRELOCITEM
 0A79:12F7       PMALLC
 0A79:4A41       PMCALLBACK
 0A79:1780       PMDOSXIRET
 0A79:1781       PMDOSXIRETD
 0A79:16D0       PMFAULTENTRYVECTOR
 0A79:1770       PMFAULTHANDLERIRET
 0A79:1774       PMFAULTHANDLERIRETD
 0000:73E8       PMFAULTVECTOR
 0A79:1339       PMFREE
 0000:6BDE       PMINT24HANDLER
 0A79:275F       PMINT2FHANDLER
 0A79:1778       PMINTHANDLERIRET
 0A79:177C       PMINTHANDLERIRETD
 0000:74E8       PMINTNO
 0A79:4F20       PMINTR13
 0A79:1A1C       PMINTR19
 0A79:507D       PMINTR25
 0A79:5135       PMINTR26
 0A79:19BB       PMINTR28
 0A79:580F       PMINTR2A
 0A79:4374       PMINTR31
 0A79:5406       PMINTR4B
 0A79:583C       PMINTR5C
 0A79:19DF       PMINTR70
 0A79:0696       PMINTRDOS
 0A79:13D0       PMINTRENTRYVECTOR
 0A79:1A1B       PMINTRIGNORE
 0A79:1BBB       PMINTRMISC
 0A79:1C71       PMINTRMOUSE
 0A79:1783       PMINTRREFLECTOR
 0A79:1AA7       PMINTRVIDEO
 0A79:136C       PMMODB
 0A79:2E70       PMRAWMODESWITCH
 0A79:2F77       PMSAVERESTORESTATE
 0000:6A74       PMUSRSP
 0000:6A76       PMUSRSS
 07F4:0C7C       POINTDEVICEHANDLER
 07F4:0006       PREVINT2FHANDLER
 07F4:000A       PREVINT69HANDLER
 0A79:3096       PUTFAULTVECTOR
 0A79:2FB0       PUTINTRVECTOR
 0A79:1A10       READCMOS
 07F4:1B90       READINIFILE
 0A79:521E       READWRITESECTORS
 0000:4748       REGCHILDCS
 0000:4746       REGCHILDIP
 0000:4742       REGCHILDSP
 0000:4744       REGCHILDSS
 0000:6BCA       REGUSERAX
 0000:6BCC       REGUSERDS
 0000:6BCE       REGUSERES
 0000:6BC8       REGUSERFL
 0000:6BC2       REGUSERSP
 0000:6BC0       REGUSERSS
 0A79:03E8       REINITGDT
 0A79:01F2       REINITIDT
 07F4:1140       RELEASELOWHEAP
 07F4:117F       RELEASEXMEMHEAP
 0A79:3420       REMOVEFREEDESCRIPTOR
 07F4:10AA       RESET286
 07F4:10B0       RESET386
 0000:7EB2       RESETSTACK
 07F4:0D6A       RESTORERMINTRVECTORS
 0A79:59F6       RESUMENETPOSTING
 0000:4780       RGBXFRBUF0
 0000:4800       RGBXFRBUF1
 0000:6BE6       RGLPFNRMISR
 0000:7E32       RGW0STACK
 0000:7D90       RGW2FSTACK
 0000:0100       RGWSTACK
 0000:7F32       RGWWOWSTACK
 0A79:1970       RM24RET
 0A79:19B9       RM24TRAP
 0A79:547F       RM4B
 07F4:1389       RMCALLBACKHOOK
 07F4:0A41       RMDEFAULTINT24HANDLER
 0000:6FE6       RMHWISR
 07F4:0E9D       RMINT2FHANDLER
 07F4:0A44       RMINTR24
 07F4:0682       RMINTRENTRYVECTOR
 07F4:0982       RMINTRREFLECTOR
 07F4:167D       RMPOSTRTN
 07F4:10E8       RMRAWMODESWITCH
 07F4:1130       RMSAVERESTORESTATE
 07F4:10D4       RMUNSIMULATEPROC
 0A79:0EEE       RSTREG
 0A79:4BD1       RZCALL
 07F4:0D4E       SAVERMINTRVECTORS
 0000:7970       SEGCURRENTHOSTDATA
 07F4:0000       SEGDXCODE
 0A79:0002       SEGDXCODEPM
 07F4:0002       SEGDXDATA
 0A79:0004       SEGDXDATAPM
 0000:470E       SEGGDT
 0000:471A       SEGIDT
 0000:4734       SEGPSP
 0000:4738       SEGPSPCHILD
 0000:796E       SELCURRENTHOSTDATA
 07F4:0004       SELDGROUP
 0A79:0000       SELDGROUPPM
 0000:472C       SELDOSSCR
 0000:4708       SELEHSTACK
 0000:4710       SELGDT
 0000:470C       SELGDTFREE
 0000:7A56       SELHEAPSTART
 0000:7A64       SELHIHEAPSTART
 0000:471C       SELIDT
 0000:7A66       SELLOWHEAPSTART
 0A79:3113       SELOFF2SEGOFF
 0000:4736       SELPSP
 0000:473A       SELPSPCHILD
 0A79:3156       SETSEGMENTADDRESS
 0A79:4101       SETUPDATADESCRIPTORS
 07F4:212E       SETUPHIMEMDRIVER
 0000:6918       SMRTDRVDELTA
 0000:691B       SMRTDRVNAME
 0A79:3FC2       SPLITBLOCK
 07F4:000E       START
 07F4:27E1       STRCMPI
 07F4:27D5       STRCPY
 0A79:36C9       STRUCTUREHEAP
 0000:4751       SYSTSS
 0A79:5DD0       SZFAULTMESSAGE
 0A79:5E08       SZRING0FAULTMESSAGE
 07F4:16F0       TERMINATEOEM
 0A79:13C5       TERMINATEPROCESS
 07F4:162F       TERMNETMAPPER
 07F4:283C       TOUPPER
 0A79:5C70       UPDATENCB
 0A79:28FE       VCD_PM_SVC_CALL
 0000:755F       WOW16BITHANDLERS
 0A79:1EE3       WOW16TRANSITIONTOUSERMODE
 0A79:24FD       WOW32INTR16REFLECTOR
 0A79:1EFD       WOW32INTRREFL
 0A79:1EEF       WOW32TRANSITIONTOUSERMODE
 0000:755D       WOWTRANSITIONTOUSERMODE
 0A79:117C       XFRFLG
 0A79:1A3B       XMSCONTROL
 0A79:29FA       XMSFUNC

  Address         Publics by Value

 0000:0100       RGWSTACK
 0000:0100       BREFLSTACK
 0000:4700       PBHWINTRSTACK
 0000:4702       PBREFLSTACK
 0000:4704       NPEHSTACKLIMIT
 0000:4706       NPEHSTACKLET
 0000:4708       SELEHSTACK
 0000:470A       CDSCGDTMAX
 0000:470C       SELGDTFREE
 0000:470E       SEGGDT
 0000:4710       SELGDT
 0000:4712       BPGDT
 0000:4712       BPGDTCB
 0000:4714       BPGDTBASE
 0000:4718       CDSCIDTMAX
 0000:471A       SEGIDT
 0000:471C       SELIDT
 0000:471E       BPIDT
 0000:471E       BPIDTCB
 0000:4720       BPIDTBASE
 0000:4724       BPRMIVT
 0000:472C       SELDOSSCR
 0000:472E       LPFNXMSFUNC
 0000:4732       IDCPUTYPE
 0000:4734       SEGPSP
 0000:4736       SELPSP
 0000:4738       SEGPSPCHILD
 0000:473A       SELPSPCHILD
 0000:473C       DTASEGMENT
 0000:473E       DTASELECTOR
 0000:4740       DTAOFFSET
 0000:4742       REGCHILDSP
 0000:4744       REGCHILDSS
 0000:4746       REGCHILDIP
 0000:4748       REGCHILDCS
 0000:474A       HMEMDOSX
 0000:474C       FFAULTABORT
 0000:474D       EXITCODE
 0000:4750       FUSINGHMA
 0000:4751       SYSTSS
 0000:477D       HIGHESTDXSEL
 0000:4780       RGBXFRBUF0
 0000:4800       RGBXFRBUF1
 0000:6800       NPXFRBUF0
 0000:6802       NPXFRBUF1
 0000:6904       EXEC_PAR_BLK
 0000:6912       FHEXEFILE
 0000:6914       CLPRELOCITEM
 0000:6916       PLPRELOCITEM
 0000:6918       SMRTDRVDELTA
 0000:691B       SMRTDRVNAME
 0000:6A74       PMUSRSP
 0000:6A76       PMUSRSS
 0000:6BC0       REGUSERSS
 0000:6BC2       REGUSERSP
 0000:6BC8       REGUSERFL
 0000:6BCA       REGUSERAX
 0000:6BCC       REGUSERDS
 0000:6BCE       REGUSERES
 0000:6BD4       LPFNUSERMOUSEHANDLER
 0000:6BDA       LPFNUSERPOINTINGHANDLER
 0000:6BDE       PMINT24HANDLER
 0000:6BE6       RGLPFNRMISR
 0000:6FE6       RMHWISR
 0000:73E6       FHARDWAREINTMOVED
 0000:73E8       PMFAULTVECTOR
 0000:74E8       PMINTNO
 0000:755D       WOWTRANSITIONTOUSERMODE
 0000:755F       WOW16BITHANDLERS
 0000:796C       CDPMICLIENTS
 0000:796E       SELCURRENTHOSTDATA
 0000:7970       SEGCURRENTHOSTDATA
 0000:7972       DPMISEGATTR
 0000:7974       DPMIFLAGS
 0000:799D       A20ENABLECOUNT
 0000:79A1       F286_287
 0000:79A6       HIGHESTSEL
 0000:79A8       FASTBOP
 0000:7A40       CKBINITIALHEAPSIZE
 0000:7A42       DSEGCURRENT
 0000:7A44       HMEMHEAP
 0000:7A52       CBHEAPSIZE
 0000:7A56       SELHEAPSTART
 0000:7A64       SELHIHEAPSTART
 0000:7A66       SELLOWHEAPSTART
 0000:7A6D       HMEM_XMS_TABLE
 0000:7A8D       HMEM_XMS_COUNT
 0000:7A8F       NOASYNCSWITCHING
 0000:7A90       LOWMEMALLOCFN
 0000:7A94       LOWMEMFREEFN
 0000:7AA0       I31HWRESET
 0000:7AAB       I31_SELECTORBITMAP
 0000:7B80       DEBUG_REGS
 0000:7BC0       FMEMM_DISABLED
 0000:7BC1       MEMM_STATE
 0000:7BC2       MEMM_CALL
 0000:7BD0       BDMASERVICEBIT
 0000:7BE4       HCB_LIST
 0000:7C90       FDEBUG
 0000:7CB8       NETHEAPSIZE
 0000:7CC6       INT28FILTER
 0000:7CD9       FASTERMODESWITCH
 0000:7CEB       FWIN30COMMDRV
 0000:7CF3       LMAIDT
 0000:7CF7       LMAGDT
 0000:7CFB       LMADXPMCODE
 0000:7D90       RGW2FSTACK
 0000:7E32       RGW0STACK
 0000:7EB2       RESETSTACK
 0000:7F32       RGWWOWSTACK
 07F4:0000       SEGDXCODE
 07F4:0002       SEGDXDATA
 07F4:0004       SELDGROUP
 07F4:0006       PREVINT2FHANDLER
 07F4:000A       PREVINT69HANDLER
 07F4:000E       START
 07F4:0141       DOSXTERMINATIONHANDLER
 07F4:0222       CHILDTERMINATIONHANDLER
 07F4:02A1       DISPLAYERRORMSG
 07F4:02BE       DETERMINEFREEMEMORY
 07F4:02D6       GOINGTODOS
 07F4:02D7       BACKFROMDOS
 07F4:0682       RMINTRENTRYVECTOR
 07F4:0982       RMINTRREFLECTOR
 07F4:0982       ENDRMINTRENTRY
 07F4:0A41       RMDEFAULTINT24HANDLER
 07F4:0A44       RMINTR24
 07F4:0C1B       MOUSEINTERRUPTHANDLER
 07F4:0C7C       POINTDEVICEHANDLER
 07F4:0D4E       SAVERMINTRVECTORS
 07F4:0D6A       RESTORERMINTRVECTORS
 07F4:0DD0       DPMI_CLIENT_PMODE_ENTRY
 07F4:0E9D       RMINT2FHANDLER
 07F4:0F90       ENTERPROTECTEDMODE
 07F4:1025       ENTERREALMODE
 07F4:10AA       RESET286
 07F4:10B0       RESET386
 07F4:10C8       LCODESEGLOC
 07F4:10D4       RMUNSIMULATEPROC
 07F4:10E8       RMRAWMODESWITCH
 07F4:1130       RMSAVERESTORESTATE
 07F4:1140       RELEASELOWHEAP
 07F4:117F       RELEASEXMEMHEAP
 07F4:1389       RMCALLBACKHOOK
 07F4:1550       EMMENABLE
 07F4:162F       TERMNETMAPPER
 07F4:167D       RMPOSTRTN
 07F4:16F0       TERMINATEOEM
 07F4:1700       CODEEND
 07F4:1700       ER_CPUTYPE
 07F4:176E       ER_PROTMODE
 07F4:17FD       ER_NOHIMEM
 07F4:1895       ER_DXINIT
 07F4:1904       ER_REALMEM
 07F4:1971       ER_EXTMEM
 07F4:19DA       ER_NOEXE
 07F4:1AAF       EMMDISABLE
 07F4:1B90       READINIFILE
 07F4:1DEC       FINDFILE
 07F4:1EF4       GETENV
 07F4:1F50       INITDOSEXTENDER
 07F4:207F       ALLOCATEEXTMEM
 07F4:212E       SETUPHIMEMDRIVER
 07F4:2183       MOVEDOSEXTENDER
 07F4:21EF       MOVEDSCRTABLES
 07F4:2285       INITGLOBALDSCRTABLE
 07F4:249B       INITINTRDSCRTABLE
 07F4:263D       INITTASKSTATESEG
 07F4:2661       CHECKCPUTYPE
 07F4:276C       GETEXENAME
 07F4:2799       PARSECOMMANDLINE
 07F4:27D5       STRCPY
 07F4:27E1       STRCMPI
 07F4:283C       TOUPPER
 0A79:0000       SELDGROUPPM
 0A79:0002       SEGDXCODEPM
 0A79:0004       SEGDXDATAPM
 0A79:0006       DXPMINIT
 0A79:01F2       REINITIDT
 0A79:03E8       REINITGDT
 0A79:042D       ALLOCATEEXCEPTIONSTACK
 0A79:0696       PMINTRDOS
 0A79:0894       LEAVEDOSEXTENDER
 0A79:08C3       DOSXIRET
 0A79:08C4       DOSENTRY
 0A79:09AE       MOVDAT
 0A79:0A14       DOSEXIT
 0A79:0B1A       IOCTLENTER
 0A79:0CD0       IOCTLEXIT
 0A79:0DCD       DOSEXITCALL
 0A79:0E7B       NET5FENTER
 0A79:0EAE       NET5FEXIT
 0A79:0EEE       RSTREG
 0A79:0F09       GTAREA
 0A79:1049       GETENTRYCD
 0A79:108D       CHECKSTATUS
 0A79:10B9       DOSXEC
 0A79:117C       XFRFLG
 0A79:1196       DFGETINTRVECTOR
 0A79:11BC       DFSETINTRVECTOR
 0A79:12F7       PMALLC
 0A79:1339       PMFREE
 0A79:136C       PMMODB
 0A79:13C5       TERMINATEPROCESS
 0A79:13D0       PMINTRENTRYVECTOR
 0A79:16D0       PMFAULTENTRYVECTOR
 0A79:1770       PMFAULTHANDLERIRET
 0A79:1774       PMFAULTHANDLERIRETD
 0A79:1778       PMINTHANDLERIRET
 0A79:177C       PMINTHANDLERIRETD
 0A79:1780       PMDOSXIRET
 0A79:1781       PMDOSXIRETD
 0A79:1783       PMINTRREFLECTOR
 0A79:1970       RM24RET
 0A79:19B9       RM24TRAP
 0A79:19BB       PMINTR28
 0A79:19DF       PMINTR70
 0A79:1A10       READCMOS
 0A79:1A1B       PMINTRIGNORE
 0A79:1A1C       PMINTR19
 0A79:1A3B       XMSCONTROL
 0A79:1AA7       PMINTRVIDEO
 0A79:1AF4       INTENTRYVIDEO
 0A79:1B48       INTEXITVIDEO
 0A79:1BBB       PMINTRMISC
 0A79:1C08       INTENTRYMISC
 0A79:1C27       INTEXITMISC
 0A79:1C71       PMINTRMOUSE
 0A79:1CBE       INTENTRYMOUSE
 0A79:1D20       INTEXITMOUSE
 0A79:1D53       ENTERINTHANDLER
 0A79:1DD1       LEAVEINTHANDLER
 0A79:1EE3       WOW16TRANSITIONTOUSERMODE
 0A79:1EEF       WOW32TRANSITIONTOUSERMODE
 0A79:1EFD       WOW32INTRREFL
 0A79:24FD       WOW32INTR16REFLECTOR
 0A79:275F       PMINT2FHANDLER
 0A79:28FE       VCD_PM_SVC_CALL
 0A79:2903       FNQUERYDOSEXTENDER
 0A79:290F       FNABORT
 0A79:29FA       XMSFUNC
 0A79:2C40       DPMISIZEINIT
 0A79:2E70       PMRAWMODESWITCH
 0A79:2F77       PMSAVERESTORESTATE
 0A79:2F8B       GETINTRVECTOR
 0A79:2FB0       PUTINTRVECTOR
 0A79:3080       GETFAULTVECTOR
 0A79:3096       PUTFAULTVECTOR
 0A79:30DB       GTPARA
 0A79:3113       SELOFF2SEGOFF
 0A79:312E       LMA2SEGOFF
 0A79:313C       GETSEGMENTADDRESS
 0A79:3156       SETSEGMENTADDRESS
 0A79:31A1       NSETSEGMENTACCESS
 0A79:31FC       NSETSEGMENTLIMIT
 0A79:3244       NSETSEGMENTBASE
 0A79:329F       NMOVEDESCRIPTOR
 0A79:3313       NWOWSETDESCRIPTOR
 0A79:3355       PARATOLDTSELECTOR
 0A79:336C       FARPARATOLDTSELECTOR
 0A79:3370       ALLOCATELDTSELECTOR
 0A79:3378       ALLOCATESELECTOR
 0A79:33AB       ALLOCATESELECTORBLOCK
 0A79:3420       REMOVEFREEDESCRIPTOR
 0A79:3463       ISSELECTORFREE
 0A79:347A       FREESELECTOR
 0A79:34B9       FREESELECTORBLOCK
 0A79:34CA       FINDLOWSELECTOR
 0A79:34DB       FINDSELECTOR
 0A79:3522       DUPSEGMENTDSCR
 0A79:3545       NSETSEGMENTDSCR
 0A79:35CF       MAKELOWSEGMENT
 0A79:35EE       PARATOLINEAR
 0A79:35F9       MOVEMEMBLOCK
 0A79:3640       INITLOWHEAP
 0A79:3641       ADDTOXMEMHEAP
 0A79:36C8       INITXMEMHEAP
 0A79:36C9       STRUCTUREHEAP
 0A79:3765       ADDSELECTORTOCHAIN
 0A79:37A4       ALLOCATEXMEM32
 0A79:37C7       FREEXMEM32
 0A79:3845       ALLOCATELOWBLOCK
 0A79:39B2       FREELOWBLOCK
 0A79:3A4E       ALLOCATEXMEMBLOCK
 0A79:3BD4       FREEXMEMBLOCK
 0A79:3C64       MODIFYXMEMBLOCK
 0A79:3DEB       CALCULATEMAXIMUMSEGMENTSPACE
 0A79:3E39       CALCULATEMAXIMUMSPACE
 0A79:3EAD       COMBINEFREEBLOCKS
 0A79:3F10       FINDFREEBLOCK
 0A79:3F9B       FREESPACE
 0A79:3FC2       SPLITBLOCK
 0A79:40BE       DISPOSEBLOCK
 0A79:4101       SETUPDATADESCRIPTORS
 0A79:4212       FREEMEMBYOWNER
 0A79:4374       PMINTR31
 0A79:4460       I31_SUCCESS
 0A79:4462       I31_PAGESIZE
 0A79:446E       I31_ALLOCSEL
 0A79:44A7       I31_FREESEL
 0A79:44F9       I31_MAPSEG2SEL
 0A79:450C       I31_GETSELINCR
 0A79:4514       I31_GETSEGADDR
 0A79:453A       I31_SETSEGADDR
 0A79:455C       I31_SETLIMIT
 0A79:45A6       I31_SETACCESS
 0A79:45D5       I31_CREATEDATAALIAS
 0A79:460B       I31_GETSETDESCRIPTOR
 0A79:46AB       I31_SPECIFICSEL
 0A79:46D2       I31_ALLOCDOSMEM
 0A79:4706       I31_FREEDOSMEM
 0A79:4724       I31_SIZEDOSMEM
 0A79:4731       I31_GETSETRMINT
 0A79:47CC       I31_GETSETFAULTVECTOR
 0A79:47FD       I31_GETSETPMINT
 0A79:483F       I31_RMCALL
 0A79:4914       I31_ALLOCCALLBACK
 0A79:4976       I31_FREECALLBACK
 0A79:4A41       PMCALLBACK
 0A79:4A8E       I31_GETFREEMEM
 0A79:4AB9       I31_ALLOCMEM
 0A79:4AF9       I31_FREEMEM
 0A79:4B29       I31_SIZEMEM
 0A79:4B6B       I31_VIRTUALINT
 0A79:4B8B       I31_VERSION
 0A79:4BA3       I31_MEMGETHEADER
 0A79:4BD1       RZCALL
 0A79:4CA7       DD_I31_SET_WATCHPOINT
 0A79:4D63       DD_I31_CLEAR_WATCHPOINT
 0A79:4DD7       DD_I31_GET_STATUS
 0A79:4E10       DD_I31_RESET_WATCHPOINT
 0A79:4E67       I31_GETSTATESAVERESTORE
 0A79:4E9B       I31_GETRAWMODESWITCH
 0A79:4ECA       I31_WOW_ALLOCSEL
 0A79:4EE8       I31_WOW_SETDESCRIPTOR
 0A79:4F03       I31_WOW_SETALLOCFUNCTIONS
 0A79:4F20       PMINTR13
 0A79:5004       INTENTRY13
 0A79:503E       INTEXIT13
 0A79:507D       PMINTR25
 0A79:5135       PMINTR26
 0A79:51ED       INTENTRY2X
 0A79:5217       INTEXIT2X
 0A79:521E       READWRITESECTORS
 0A79:5406       PMINTR4B
 0A79:547F       RM4B
 0A79:55D0       INITNETMAPPER
 0A79:580F       PMINTR2A
 0A79:583C       PMINTR5C
 0A79:5911       NETBIOSPOSTROUTINE
 0A79:59DF       DELAYNETPOSTING
 0A79:59F6       RESUMENETPOSTING
 0A79:5ABF       COPYBUFFEROUT
 0A79:5AE9       COPYBUFFER
 0A79:5BD7       DELINK
 0A79:5C0F       FINDTARGETNCB
 0A79:5C52       GETENTRYEXITFLAGS
 0A79:5C70       UPDATENCB
 0A79:5CB0       HANDLENETBIOSANR
 0A79:5D95       HOOKNETBIOSHWINT
 0A79:5DC0       INITIALIZEOEM
 0A79:5DD0       SZFAULTMESSAGE
 0A79:5E08       SZRING0FAULTMESSAGE
 0A79:5E30       NPXEXCEPTIONHANDLER
 0A79:5EEC       ENDNPXEXCEPTIONHANDLER
 0A79:5EF0       CODEENDPM

Program entry point at 07F4:000E
